:1000000012C0189518951895189518951895189563
:100010001895189518951895189518951895189578
:100020001895189518958FE58DBFC8E3E0E24E2E20
:1000300084E08EBFD4E0F4E05F2EA89584B7082E4C
:10004000877F84BF88E1992781BD91BDEEEFF3E002
:10005000A0E6B0E088278D933197E9F7E4D36624D2
:10006000A298A398889889988A988B989A9A9B9A2C
:10007000809A819A829A839A70EF71BB7FE072BBFB
:1000800073E074BB7CE075BB26D688E0809361008A
:1000900088E08093620088E180936B00ACE6B0E07A
:1000A000E8E4FDE04BD480E2809363008AE580932E
:1000B000640080EC8093650080EE8093660080E8A9
:1000C0008093670080EA8093680087E680936900E8
:1000D00087E780936A00EEEEF0E088E6ECD358E024
:1000E000C895802DE2D331965A95D1F704C01B1BD9
:1000F0001B1B1B1B1B207DD38CE0DDD37AD3E0E5DB
:10010000FDE071D38FEB11E083D3E2E6FDE06BD32A
:10011000E2E0F0E07FD36DD318E81E7FE1D5F7D59C
:1001200010916300F4D5EAD518E81E7FD9D5EFD534
:1001300010916800ECD5E2D518E81E7FD1D5E7D53F
:1001400010916700E4D5DAD518E81E7FC9D5DFD550
:1001500010916600DCD5D2D518E81E7FC1D5D7D561
:1001600010916500D4D5CAD518E81E7FB9D5CFD572
:1001700010916A00CCD5C2D518E81E7FB1D5C7D57D
:1001800010916900C4D5BAD518E81E7FA9D5BFD58E
:1001900010916400BCD5B2D5829904C085E090E08E
:1001A000B6D3D5D0839904C085E090E0B0D363D1B5
:1001B000809904C085E090E0AAD3EFD1819904C072
:1001C00085E090E0A4D37DD29A9904C085E090E0C8
:1001D0009ED309D09B9904C085E090E098D349D084
:1001E000DBCFF894FFCF009163000F3308F036C0E7
:1001F000A3E6B0E08C918F5F8C93ECE4FDE020D51A
:10020000E3E6F0E0D080EE24FF24002734D46BD462
:10021000EDE0F0E0A4E7B0E099D300E110E00F9347
:100220001F93E4E7F0E018D5EDE0F0E0CCD3E4E193
:10023000F0E0EE0C000FE7944D2D5E2D1F910F9115
:10024000041B150BA2E7B0E00D931C9318E81E7F6A
:1002500047D55DD5109163005AD550D58FE711E091
:10026000D7D2E4E7FDE0BFD24CD084E190E04FD399
:10027000089500916300003010F009F001C036C00D
:1002800080916300815080936300ECE4FDE0D8D45A
:10029000E3E6F0E0D080EE24FF240027ECD323D463
:1002A000EDE0F0E0A4E7B0E051D300E110E00F93FF
:1002B0001F93E4E7F0E0D0D4EDE0F0E084D3E4E194
:1002C000F0E0EE0C000FE7944D2D5E2D1F910F9185
:1002D000041B150BA2E7B0E00D931C9318E81E7FDA
:1002E000FFD415D51091630012D508D58FE711E022
:1002F0008FD2E4E7FDE077D204D084E190E007D329
:1003000008958FEB11E084D281E080937100009119
:100310007100003110F009F019C0A2E7B0E04D9172
:100320005C91A1E7B0E00D9111270417150710F0BB
:1003300009F003C085E0B9D202C080E2B6D2A1E7DD
:10034000B0E08C918F5F8C9308F4E1CF0895A2E622
:10035000B0E08C918F5F8C93009162000F3010F0B1
:1003600009F001C003C08FE0809362000091620039
:10037000013009F004C080E68093690061C002305A
:1003800009F004C081E6809369005AC0033009F087
:1003900004C082E68093690053C0043009F004C0B1
:1003A00083E6809369004CC0053009F004C084E600
:1003B0008093690045C0063009F004C085E680934B
:1003C00069003EC0073009F004C086E680936900EA
:1003D00037C0083009F004C087E68093690030C058
:1003E000093009F004C08EE68093690029C00A3004
:1003F00009F004C08DE68093690022C00B3009F03B
:1004000004C08CE6809369001BC00C3009F004C066
:100410008BE68093690014C00D3009F004C08AE6B1
:10042000809369000DC00E3009F004C089E6809306
:10043000690006C00F3009F003C088E680936900A8
:1004400018E81E7F4DD463D41091690060D456D44F
:10045000A2E6B0E08C91A2E7B0E08D9388278C9360
:100460008FE711E0D5D1E6E8FDE0BDD14ADF88ECA9
:1004700090E04DD208958091620081508093620097
:1004800000916200013008F003C081E080936200B7
:1004900000916200013009F004C080E68093690099
:1004A00061C0023009F004C081E6809369005AC03F
:1004B000033009F004C082E68093690053C0043021
:1004C00009F004C083E6809369004CC0053009F050
:1004D00004C084E68093690045C0063009F004C07A
:1004E00085E6809369003EC0073009F004C086E6C7
:1004F0008093690037C0083009F004C087E6809314
:10050000690030C0093009F004C08EE680936900AC
:1005100029C00A3009F004C08DE68093690022C02A
:100520000B3009F004C08CE6809369001BC00C30CE
:1005300009F004C08BE68093690014C00D3009F007
:1005400004C08AE6809369000DC00E3009F004C033
:1005500089E68093690006C00F3009F003C088E681
:100560008093690018E81E7FBBD3D1D31091690036
:10057000CED3C4D3A2E6B0E08C91A2E7B0E08D93D5
:1005800088278C938FE711E043D1E6E8FDE02BD17B
:10059000B8DE88EC90E0BBD10895A1E6B0E08C9184
:1005A0008F5F8C93009161000F3010F009F001C053
:1005B00003C08FE08093610000916100013009F079
:1005C00004C080E780936A0061C0023009F004C073
:1005D00081E780936A005AC0033009F004C082E7C3
:1005E00080936A0053C0043009F004C083E780930D
:1005F0006A004CC0053009F004C084E780936A00AB
:1006000045C0063009F004C085E780936A003EC00B
:10061000073009F004C086E780936A0037C00830CD
:1006200009F004C087E780936A0030C0093009F000
:1006300004C08EE780936A0029C00A3009F004C024
:100640008DE780936A0022C00B3009F004C08CE76C
:1006500080936A001BC00C3009F004C08BE78093C4
:100660006A0014C00D3009F004C08AE780936A0064
:100670000DC00E3009F004C089E780936A0006C0FF
:100680000F3009F003C088E780936A0018E81E7FE6
:1006900027D33DD310916A003AD330D3A1E6B0E01E
:1006A0008C91A2E7B0E08D9388278C938FE711E0BF
:1006B000AFD0E8E9FDE097D024DE88EC90E027D1C8
:1006C00008958091610081508093610000916100E4
:1006D000013008F003C081E0809361000091610067
:1006E000013009F004C080E780936A0061C00230E5
:1006F00009F004C081E780936A005AC0033009F012
:1007000004C082E780936A0053C0043009F004C03B
:1007100083E780936A004CC0053009F004C084E789
:1007200080936A0045C0063009F004C085E78093D5
:100730006A003EC0073009F004C086E780936A0073
:1007400037C0083009F004C087E780936A0030C0E2
:10075000093009F004C08EE780936A0029C00A308E
:1007600009F004C08DE780936A0022C00B3009F0C5
:1007700004C08CE780936A001BC00C3009F004C0F1
:100780008BE780936A0014C00D3009F004C08AE73B
:1007900080936A000DC00E3009F004C089E7809391
:1007A0006A0006C00F3009F003C088E780936A0032
:1007B00018E81E7F95D2ABD210916A00A8D29ED2C3
:1007C000A1E6B0E08C91A2E7B0E08D9388278C93EE
:1007D0008FE711E01DD0E8E9FDE005D092DD88EC5F
:1007E00090E095D00895A2D0802D11F05ED0FBCF7F
:1007F000089581E060D014D080E85DC08FE721309B
:1008000039F08FEB223021F08FE8233009F08FECA4
:10081000810F51C088EE93E07AD03197D9F70895CF
:1008200083E0992774C08AEF90E071D08D9AB89ACE
:100830008E9A8F9AB99ABA9AC29885E090E067D05A
:10084000C1989598C098969A979AC19AEF93FF93FA
:10085000E4ECF0E050D0FF91EF91C19855D0C19AEF
:10086000EF93FF93E4ECF0E046D0FF91EF91C19855
:100870004BD0C19AEF93FF93E4ECF0E03CD0FF91B2
:10088000EF91C19841D09798C19AEF93FF93E4EC10
:10089000F0E031D0FF91EF91C19836D088E20BD0D3
:1008A0008EE009D086E007D00895C29A829505D0DF
:1008B00004D02AD00895C298F9CF859510F4979A5C
:1008C00001C09798859510F4969A01C096988595E1
:1008D00010F4C09A01C0C098859510F4959A01C093
:1008E0009598C19AEF93FF93E4ECF0E004D0FF9168
:1008F000EF91C19808953197F1F70895689462F8DF
:100900000895E89462F8089581E090E000C0EF93C4
:10091000FF93EE27E82BE92B31F0E0EDF7E031977C
:10092000F1F70197D1F7FF91EF910895C8953196AE
:100930000020089591E005C092E003C094E001C05A
:1009400098E0F4DF0D929A95E1F7089594E0819193
:100950008D939A95E1F70895B7FE089590E8B9163A
:1009600011F4D0FE08959FEFD91AE90AF90A09F4A3
:10097000039508950F928F939F93D216E306F40682
:100980000FB680E890E8802795270FBE890739F0D9
:100990000FB6892B87FD02C081E008260FBE9F910C
:1009A0008F910F900895D190E190F1900191089569
:1009B00021913191419151910895502F2D2D3E2D2E
:1009C0004F2D612F0895EFDF992711278F2D880F65
:1009D00080E8F82A802F881F08F41FEF41F08F5716
:1009E000082F07FD04C0003240F08FEF01C08827B8
:1009F000982FD82EE82EF82E09C08FE1801B082FE3
:100A0000F694E794D79497950A95D1F7112351F06E
:100A10009095D094E094F09481E0980F8827D81EA8
:100A2000E81EF81E0F2DFE2CED2CD92E0895D09423
:100A3000E094F09491E0D90E9927E91EF91E1095E3
:100A40000895652F90E8440F551F5927990F479532
:100A50006078102F90E8FF0C001F0927990FF7947A
:100A6000107800380895FF0C90E89027110F9795A3
:100A7000F794092F0895102FBD2CDE2CEF2CF02EAB
:100A800011234AF4B094D094E094F0949FEFB91AF3
:100A9000D90AE90AF90A0EE1FF2039F4FE2CED2CFF
:100AA000DB2CBB240850C2F752C032F00A95BB0CB5
:100AB000DD1CEE1CFF1CF9CF4FDFD5CF2DEC3CEC3D
:100AC0004CEC5DE366270FC06EDF77DFDD24EE249C
:100AD00090E8F92E0FE307C06BDF05C0222733270C
:100AE00040E251E46627552351F1002381F1A9DF4B
:100AF00071F11627005850580894050B18F407FD9B
:100B000003C025C007FD23C0469537952795F69469
:100B1000E794D79422D0FF202AF0DD0CEE1CFF1CB6
:100B2000015073F09D2D969548F0DD203AF4EE20AB
:100B30002AF491E0D90E9927E91EF91E94CF07C037
:100B40009FE7092FF92A9FEFD92EE92E0895DD247A
:100B5000EE24FF240027112708959F929924AA24A8
:100B6000BB2488E1D216E306F40628F0D21AE30A81
:100B7000F40A089401C08894991CAA1CBB1CDD0CC3
:100B8000EE1CFF1C8A9571F7D92CEA2CFB2C9F9048
:100B900008950AF045D067CF5FE322273327442723
:100BA00001C006DF4EDF5038B1F3003899F3902FC3
:100BB000951B8BF312F434D0FACF983118F022271A
:100BC00033274427983028F0232F342F4427985078
:100BD000F9CF992329F04695379527959A95D9F716
:100BE000912F962742F014D0B0F6F794E794D7945B
:100BF0000F5F8BF6A5CF10D051F008F418DFFF205F
:100C000052F2DD0CEE1CFF1C0150CBF799CF9FCFA9
:100C1000D20EE31EF41E0895D21AE30AF40A0895D0
:100C2000DF92EF92FF920F931F93D22EE32EF42EBA
:100C3000052F162F6F915F914F913F912F9108953E
:100C400075DE202D73DE302D71DE402D6FDE502DD0
:100C50000895A9DE80E003C0A6DE802F8078882377
:100C600021F0DF92EF92FF920F938F93EADE802FB5
:100C7000839512F46CDF1BC080958A95885E0AF418
:100C800015C088501AF40CD0D92210C0DD24885029
:100C90001AF406D0E9220AC0EE2402D0F92206C0D6
:100CA0009FEF8770990F8A95EAF70895DCDE8F91A0
:100CB0008823D9F35F914F913F912F910F935ADE83
:100CC0000F9199F390F302D050686CCF5FE340E846
:100CD000332722270895A498A598AC98AD98089535
:100CE000A59AA49803D0A59801D0A49AEF93FF9356
:100CF000E0E1F0E000DEFF91EF910895A59AA49A5B
:100D0000F5DFA5989D9BFECFF1DFA498EFCF089467
:100D1000111F01C0110F69F0A59A18F40000A498E2
:100D200002C0A49A00C0E2DFA5989D9BFECFDEDF43
:100D3000F1CFA59AA498DADFA5989D9BFECFE89401
:100D40009C99689462F8D2CF0000000000007C40BB
:100D5000205444413733313320507265416D702047
:100D6000000020204C6F75646E657373204F6E20F9
:100D70002020000020202020566F6C756D652020FB
:100D80002020202000002D2020202042617373208D
:100D900020202020202B00002D20202020547265B0
:0A0DA000626C65202020202B00006B
:00000001FF
